:020000000528D1
:10000800F1298B13831203138312031385018601CD
:100018008316FF30831603138500FF308600831292
:100028008B13063083120313A000A101A2018730AD
:1000380083168316031381008312C33083120313BC
:10004800CE00CF018100A0308B00D001FF30D3015A
:10005800D401D700D800D501D601D900DA00CF28BD
:1000680083120313D2000310500D533E84008313F0
:1000780051088000840A52088000D00A5008023AC9
:100088000319D0010310500D8313533E8400000858
:10009800840A000403194128801B412800088A00AB
:1000A800840300088200831203134108C500400836
:1000B800023E0318C50A83134518831784000008F5
:1000C800C2004108C5004008013E0318C50A831351
:1000D80045188317840000084206031974287F28EE
:1000E80083120313BD010130FF3ABD09013E031914
:1000F800BD0ABC00B12883120313C50103304207AF
:100108000318C50A4007C4000318C50A4108C507F3
:10011800831345188317440884000008C300C20AE3
:10012800831341188317400884000008420203180B
:100138009E28A12883120313C2014108C500400864
:10014800023E0318C50A8313451883178400420822
:100158008000BD014308BC00B128831203133F0887
:100168008A003E088200FF3083120313C007031879
:10017800C10AFF30C1074208C0070318C10A430873
:10018800C1070730C005C101C00A0319C10A3F08E9
:100198008A003E088200831203138501FE3083160D
:1001A80003138500831203138601FF30831603139C
:1001B80086000730831203139F000130B500013019
:1001C8008400840753308407831399308000840A9D
:1001D800033080005008013A031DF3284128031119
:1001E8000319F728F828EB29831203138501B401B2
:1001F8003508B8000310B80D3808FF3EB8003408B9
:10020800803AFC003808803A7C02031C0C29332908
:1002180083120313D2010430D100500884008407EC
:10022800573084078313840A801784035108800099
:10023800840A520880002430D10001303428412833
:1002480083120313500884008407573084078313EC
:10025800840A801F232901308506B40AFC288312EA
:100268000313D2011330D10050088400840757309B
:1002780084078313840A8017840351088000840A42
:10028800520880004B30D1000130342841288312B5
:100298000313500884008407573084078313840AA3
:1002A800801F4A29031103195A295B29EA29831255
:1002B8000313C1012030C0000130BF006830BE0008
:1002C80000308A0057308200831203133D08B700BC
:1002D8003C08B6000310B71F0314031C74297529C2
:1002E800EA29831203133708B90036087F39B800A2
:1002F800B9010311B91B862906303806031D862962
:100308000030390603198929B229831203133708E3
:10031800B90036088039B800B9013808390403191A
:100328009629B12983120313C101B51BC1093508E8
:10033800C000C3010130FF3AC309013E0319C30AD3
:10034800C2000130BF00AD30BE0000308A00B730B7
:100358008200831203133C08B500E92983120313B2
:100368003708B90036087F39B800B9010311B91B3D
:10037800C32907303806031DC3290030390603197D
:10038800C629E929831203133708B90036088039CA
:10039800B800B901380839040319D329E9298312A7
:1003A8000313C101B51BC1093508C000C3010130E1
:1003B800C2000130BF00E530BE0000308A00B7300F
:1003C8008200831203133C08B5005629F3288312D0
:1003D800031333088A0032088200FF00030E8312D9
:1003E800031383120313C800C80E0A08C9000408BF
:1003F800CA000B1D152A4E0881005030CF07B430B3
:100408000318013EFF3A013ECE000B11FF30D81B06
:10041800102AD707031CD807DA1B152AD907031C8B
:10042800DA077C08CB007D08CC007E08CD004D089B
:10043800FE004C08FD004B08FC004A0884004908EF
:100448008A0048088300FF0E7F0E090083160313F5
:100458002408A7002308013E0318A70AA70183134D
:1004680084000008013EA60083132418831723087C
:100478008400000826020318422A452A831603131B
:10048800A6012408A8002308023E0318A80A83131B
:10049800281883178400000826060319542A5B2AA3
:1004A800013083160313A000A009A00A872A831627
:1004B80003132408A8002308013E0318A80A83137D
:1004C800281883178400A8010008033E0318A80A07
:1004D8002307A7000318A80A2408A80783132818C5
:1004E800831727088400250880002408A80023080B
:1004F800013E0318A80A83132818831784002608C6
:100508008000A001872A8316031322088A00210885
:10051800820083120313AA01AB016308AC00AD018A
:10052800AE016408AF0063088316031385048312C1
:100538000313640883160313860404308312031319
:10054800A9006608B1006508B00062088A00610861
:1005580082008312031330083104031DB42AEA2AE7
:100568000130F000F10108307102031CBC2AEA2AAC
:10057800831203136D087005003A031DC42AE62A86
:100588007108831203136F07F2006E087005003AB2
:10059800031DCF2AD02AF2178312031331088316BA
:1005A8000313A40083120313300883160313A30054
:1005B8007208A5000230A200E630A10002308A00CD
:1005C8002A3082000310F00DF10AB72A83120313B0
:1005D8006C088A006B088200831203132C08003A07
:1005E800031DF72A1E2B831203130508E6000508CE
:1005F800E5000508E6040508E5050508E60405081C
:10060800E5052B08E4000508AB0064082B06E300A9
:100618002B08E6042B08E50566086506E40064086F
:1006280063042C05003A031D1A2B1E2B033083127A
:100638000313A9002F08003A031D232B4A2B83120A
:1006480003130608E6000608E5000608E60406089F
:10065800E5050608E6040608E5052E08E400060890
:10066800AE0064082E06E3002E08E6042E08E50511
:1006780066086506E400640863042F05003A031D54
:10068800462B4A2B033083120313A9002908003A8A
:10069800031D4F2B932BFF3083120313A90729083F
:1006A800003A0319582B932B831203132A082B069D
:1006B8002C05E3006308003A031D632B752B831296
:1006C80003132B082C05AA006308ED002A08EE0086
:1006D800EF010330EC007530EB0002308A00AD30DA
:1006E8008200831203132D082E062F05E3006308EA
:1006F800003A031D802B932B831203132E082F051A
:10070800AD006308ED002D08EE000830EF0003305F
:10071800EC009330EB0002308A00AD308200831287
:10072800031362088A0061088200C0308312031331
:10073800E300E401E6012030E5000330E200A930DF
:10074800E10002308A008D30820003110319AD2BBD
:10075800AE2BDB2B033083120313E200B830E10029
:1007680002308A00F030820083120313D101D201D3
:10077800500884008407573084078313840A80173D
:10078800840351088000840A52088000CF30D100C9
:100798000330342841288312031350088400840747
:1007A800573084078313840A801FCE2BA92B83120A
:0A07B80003135C088A005B0882004E
:02400E00103F61
:00000001FF
